:1000000000308A00482800000A108A100A1182076E
:100010000134F634F634F6340134FF34FF340A1078
:100020008A100A11820700347634763476348934A3
:10003000FF34FF340A108A100A11820781347E349B
:100040007E347E34BD34FF34FF340A108A100A1126
:10005000820700347E347E347E348134FF34FF34B2
:100060002230840083130008031947280130F80068
:10007000BF30F7006400F70B3A28F80B38284A30F5
:10008000F700F70B412800006400800B362800348D
:10009000840183131F30830583161F149F141F15BB
:1000A0009F1107309C00FF308312A00083161F149D
:1000B0009F141F159F1183121F108316091283129C
:1000C0009412A0122008831687008312201620089D
:1000D000831687008312A011200883168700013041
:1000E000831294000030831694000108C739083841
:1000F0008100831290010030F800920000308316D6
:10010000920007309C00050864000230F700F70BEE
:1001100087288A281C0883120D1383169D018312D9
:10012000A1012108063C031CA22821080420A200EA
:10013000831686018312220886000130A200302037
:10014000A10A9128A1012108063C031CB42821081A
:100150000F20A20083168601831222088600013038
:10016000A2003020A10AA328A1012108063C031CFB
:10017000C62821081A20A2008316860183122208AD
:1001800086000130A2003020A10AB528A101210873
:10019000063C031CD82821082520A20083168601CE
:1001A0008312220886000130A2003020A10AC7284D
:1001B000A1012108063C031CEA2821080420A20012
:1001C000831686018312220886000130A2003020A7
:0E01D000A10AD9288E30A200302090286300AA
:02400E00393F38
:00000001FF
